:100000000C9472000C947E000C947E000C947E0084
:100010000C947E000C947E000C947E000C947E0068
:100020000C947E000C947E000C947E000C947E0058
:100030000C947E000C947E000C947E000C947E0048
:100040000C947E000C947E000C947E000C947E0038
:100050000C947E000C947E000C947E000C947E0028
:100060000C947E000C947E000C947E000C947E0018
:100070000C947E000C947E000C947E000C947E0008
:100080000C947E000C947E000C947E000C947E00F8
:100090000C947E000C947E000C947E000C947E00E8
:1000A0000C947E000C947E000C947E000C947E00D8
:1000B0000C947E000C947E000C947E000C947E00C8
:1000C0000C947E000C947E000C947E000C947E00B8
:1000D0000C947E000C947E000C947E000C947E00A8
:1000E0000C947E0011241FBECFEFD1E2DEBFCDBF46
:1000F00000E00CBF0E9480000C94AA000C94000049
:100100008FEF87B981B914B885B981E093B192B9FD
:1001100093B19F3F69F488B9EFE1FEE43197F1F7BD
:1001200000C0000018B8EFE1FEE43197F1F70FC00E
:1001300093B19111EBCF88B9EFE3FCE93197F1F777
:1001400000C0000018B8EFE3FCE93197F1F700C0F8
:080150000000DCCFF894FFCFA2
:00000001FF
